:020000040000fa
:08000000101b040000000000c9
:020000040000fa
:10000800041a0000081a00000c1a0000101a000058
:10001800141a00000c1b00000c1b00000c1b000035
:10002800181a00001c1a0000201a0000241a0000e8
:100038000c1b0000281a00002c1a0000301a0000bf
:10004800341a0000381a00003c1a0000401a000058
:10005800441a0000481a00000c1b00000c1b00008a
:100068004c1a0000501a0000541a0000581a0000d8
:100078005c1a00000c1b0000601a0000641a0000e3
:100088000c1b0000681a00006c1a0000701a0000af
:10009800741a0000781a00007c1a0000801a000008
:1000a800841a0000881a00000c1b00000c1b0000ba
:1000b8000c1b00008c1a0000901a0000941a000013
:1000c800981a00009c1a0000a01a0000a41a000048
:1000d800a81a0000ac1a00000c1b00000c1b000042
:1000e8000c1b0000b01a0000b41a00000c1b000022
:1000f8000c1b0000b81a0000bc1a00000c1b000002
:100108000c1b00000c1b00000c1b00000c1b00004b
:100118000c1b00000c1b0000c01a00000c1b000088
:100128000c1b0000c41a0000c81a0000cc1a0000fa
:100138000c1b00000c1b00000c1b00000c1b00001b
:10014800d01a00000c1b00000c1b00000c1b000048
:100158000c1b0000d41a00000c1b00000c1b000034
:100168000c1b0000d81a0000dc1a0000e01a00007e
:10017800e41a0000e81a0000ec1a0000f01a000067
:10018800f41a0000f81a0000fc1a0000001b000016
:10019800041b0000081b00000c1b00000c1b0000c7
:1001a8000c1b00000c1b00000c1b00000c1b0000ab
:1001b8000c1b00000c1b00000c1b00000c1b00009b
:1001c8000c1b00000c1b00000c1b00000c1b00008b
:1001d8000c1b00000c1b00000c1b00000c1b00007b
:1001e8000c1b00000c1b00000c1b00000c1b00006b
:0801f8000c1b00000c1b0000b1
:020000040000fa
:04020800ec1b0000eb
:020000040000fa
:04020c00ec1b0000e7
:020000040000fa
:04021000ec1b0000e3
:020000040000fa
:04021400ec1b0000df
:020000040000fa
:04021800ec1b0000db
:020000040000fa
:04021c00ec1b0000d7
:020000040000fa
:04022000ec1b0000d3
:020000040000fa
:04022400ec1b0000cf
:020000040000fa
:04022800ec1b0000cb
:020000040000fa
:04022c00ec1b0000c7
:020000040000fa
:04023000ec1b0000c3
:020000040000fa
:04023400ec1b0000bf
:020000040000fa
:04023800ec1b0000bb
:020000040000fa
:04023c00ec1b0000b7
:020000040000fa
:04024000ec1b0000b3
:020000040000fa
:04024400ec1b0000af
:020000040000fa
:04024800ec1b0000ab
:020000040000fa
:04024c00ec1b0000a7
:020000040000fa
:04025000ec1b0000a3
:020000040000fa
:04025400ec1b00009f
:020000040000fa
:04025800ec1b00009b
:020000040000fa
:04025c00ec1b000097
:020000040000fa
:04026000ec1b000093
:020000040000fa
:04026400ec1b00008f
:020000040000fa
:04026800ec1b00008b
:020000040000fa
:04026c00ec1b000087
:020000040000fa
:04027000ec1b000083
:020000040000fa
:04027400ec1b00007f
:020000040000fa
:04027800ec1b00007b
:020000040000fa
:04027c00ec1b000077
:020000040000fa
:04028000ec1b000073
:020000040000fa
:04028400ec1b00006f
:020000040000fa
:04028800ec1b00006b
:020000040000fa
:04028c00ec1b000067
:020000040000fa
:04029000ec1b000063
:020000040000fa
:04029400ec1b00005f
:020000040000fa
:04029800ec1b00005b
:020000040000fa
:04029c00ec1b000057
:020000040000fa
:0402a000ec1b000053
:020000040000fa
:0402a400ec1b00004f
:020000040000fa
:0402a800ec1b00004b
:020000040000fa
:0402ac00ec1b000047
:020000040000fa
:0402b000ec1b000043
:020000040000fa
:0402b400ec1b00003f
:020000040000fa
:0402b800ec1b00003b
:020000040000fa
:0402bc00ec1b000037
:020000040000fa
:0402c000ec1b000033
:020000040000fa
:0402c400ec1b00002f
:020000040000fa
:0402c800ec1b00002b
:020000040000fa
:0402cc00ec1b000027
:020000040000fa
:0402d000ec1b000023
:020000040000fa
:0402d400ec1b00001f
:020000040000fa
:0402d800ec1b00001b
:020000040000fa
:0402dc00ec1b000017
:020000040000fa
:0402e000ec1b000013
:020000040000fa
:0402e400ec1b00000f
:020000040000fa
:0402e800ec1b00000b
:020000040000fa
:0402ec00ec1b000007
:020000040000fa
:0402f000ec1b000003
:020000040000fa
:0402f400ec1b0000ff
:020000040000fa
:0402f800ec1b0000fb
:020000040000fa
:0402fc00ec1b0000f7
:020000040000fa
:04030000ec1b0000f2
:020000040000fa
:04030400ec1b0000ee
:020000040000fa
:04030800ec1b0000ea
:020000040000fa
:04030c00ec1b0000e6
:020000040000fa
:04031000ec1b0000e2
:020000040000fa
:04031400ec1b0000de
:020000040000fa
:04031800ec1b0000da
:020000040000fa
:04031c00ec1b0000d6
:020000040000fa
:04032000ec1b0000d2
:020000040000fa
:04032400ec1b0000ce
:020000040000fa
:04032800ec1b0000ca
:020000040000fa
:04032c00ec1b0000c6
:020000040000fa
:04033000ec1b0000c2
:020000040000fa
:04033400ec1b0000be
:020000040000fa
:04033800ec1b0000ba
:020000040000fa
:04033c00ec1b0000b6
:020000040000fa
:04034000ec1b0000b2
:020000040000fa
:04034400ec1b0000ae
:020000040000fa
:04034800ec1b0000aa
:020000040000fa
:04034c00ec1b0000a6
:020000040000fa
:04035000ec1b0000a2
:020000040000fa
:04035400ec1b00009e
:020000040000fa
:04035800ec1b00009a
:020000040000fa
:04035c00ec1b000096
:020000040000fa
:04036000ec1b000092
:020000040000fa
:04036400ec1b00008e
:020000040000fa
:04036800ec1b00008a
:020000040000fa
:04036c00ec1b000086
:020000040000fa
:04037000ec1b000082
:020000040000fa
:04037400ec1b00007e
:020000040000fa
:04037800ec1b00007a
:020000040000fa
:04037c00ec1b000076
:020000040000fa
:04038000ec1b000072
:020000040000fa
:04038400ec1b00006e
:020000040000fa
:04038800ec1b00006a
:020000040000fa
:04038c00ec1b000066
:020000040000fa
:04039000ec1b000062
:020000040000fa
:04039400ec1b00005e
:020000040000fa
:04039800ec1b00005a
:020000040000fa
:04039c00ec1b000056
:020000040000fa
:10340000101b040000000000ec1b04000000000082
:10341000ec1b040000000000ec1b04000000000096
:10342000ec1b040000000000ec1b04000000000086
:10343000ec1b040000000000ec1b04000000000076
:10344000ec1b040000000000d81b0400000000007a
:10345000ec1b040000000000ec1b04000000000056
:10346000ec1b040000000000ec1b04000000000046
:10347000ec1b040000000000ec1b04000000000036
:10348000ec1b040000000000ec1b04000000000026
:10349000ec1b040000000000ec1b04000000000016
:1034a000ec1b040000000000ec1b04000000000006
:1034b000ec1b040000000000ec1b040000000000f6
:1034c000ec1b040000000000ec1b040000000000e6
:1034d000ec1b040000000000ec1b040000000000d6
:1034e000ec1b040000000000ec1b040000000000c6
:1034f000ec1b040000000000ec1b040000000000b6
:10350000ec1b040000000000ec1b040000000000a5
:10351000ec1b040000000000ec1b04000000000095
:10352000ec1b040000000000ec1b04000000000085
:10353000ec1b040000000000ec1b04000000000075
:10354000ec1b040000000000ec1b04000000000065
:10355000ec1b040000000000ec1b04000000000055
:10356000ec1b040000000000ec1b04000000000045
:10357000ec1b040000000000ec1b04000000000035
:10358000ec1b040000000000ec1b04000000000025
:10359000ec1b040000000000ec1b04000000000015
:1035a000ec1b040000000000ec1b04000000000005
:1035b000ec1b040000000000ec1b040000000000f5
:1035c000ec1b040000000000ec1b040000000000e5
:1035d000ec1b040000000000ec1b040000000000d5
:1035e000ec1b040000000000ec1b040000000000c5
:1035f000ec1b040000000000ec1b040000000000b5
:10360000ec1b040000000000ec1b040000000000a4
:10361000ec1b040000000000ec1b04000000000094
:020000040000fa
:10362000af8820000e7f24000e01880000000000fb
:10363000000020000000e000020032000001200035
:103640002002880014000700650007000000e00069
:1036500003003a0080ab2300010020000200370085
:103660000000200001002000810f700001003200e6
:1036700014000700000020000000e00002003200fb
:1036800000000200000000001838020000000000e6
:103690000040da000000fe004440a900600820005d
:1036a0000000e0000300320000002000a0018800bc
:1036b0004440a800000006008a1f78008b1f780095
:1036c0000000060091018800800478000000eb00f3
:1036d0001a003700e284440032a0b4009905ba0011
:1036e000e284440032a0b4009906ba00e2844400a7
:1036f00032a0b4000006eb00476fde00fd07b20009
:10370000636ce10003003a00ebff07000000eb00f0
:103710000a003700606ce10004003a00005deb0035
:103720008b05e900fdff3e00040037006168e10001
:10373000010032000086eb000b00070019c7ba0039
:103740001905ba000e04e00003003a000a00e00088
:10375000e0ff3a0000000600fe07b2009e0188006c
:103760008a047800f5ff3700395dba008b05e9005f
:103770000c003200295dba008b05e9000800320018
:103780000c00e00003003a00e284440032a0b400e0
:10379000f5ff370019ddba008b05e900faff3a00a2
:1037a0008904e800e184440032a0b400000006006f
:1037b0003400f800881f780008002000a801880065
:1037c0004f0478000000fa008460a9000080fa002d
:1037d0003400f900004006000040da000000fe005e
:1037e000000005004f89de0082017800a202370048
:1037f0006011b800b002370007f8270007836100a6
:103800000638e10004003a00f707200087836100d2
:103810008703710001003a0003f0a200889fbe00f8
:103820008a9fbe008c9fbe00470ade000480a10074
:10383000c71ade000580a100070028000785600088
:1038400087856100f70f20000720e1009e0032000d
:103850000728e1009c003200010678000400e00027
:10386000b4003200f7072000878060000170a000dc
:103870000500e000c0003200f707200087816100ea
:103880000370a000050652000f003a000b50e10043
:103890000b0032000308e10002003a000200e100e0
:1038a0007e0032000204500083845800040031007e
:1038b0000001fd008101fd008402fd008a05fd007c
:1038c0006044b800210037000520e10005003d00fc
:1038d0000001fd008101fd008402fd008a05fd005c
:1038e000050652007a60e100050035000170a10074
:1038f0004722dd00848070008a80700063003700fa
:103900006044b800ef02660007ff2f00070666005c
:103910000500e00006003400f08312008714dd008b
:103920000511de00071bdd00060171008519de00b0
:103930007060e10005003500090478008204780019
:10394000030178008001eb00700656000b50e10087
:1039500003003a0002004000838048000400370062
:1039600060041400e0841c000200580083805800aa
:103970000188a300060032008100d1000080d3003e
:103980008984d3000884d3000402e80027003700ac
:103990000178a30025003a000100e0000300320096
:1039a0008186cf00698656000a0037008c0020000f
:1039b0000000e00004003a00090078008804780064
:1039c0000004eb00700252008086cf000d06460016
:1039d0000c06e9007060e100060035008000780008
:1039e00009007800880478000004eb007006560097
:1039f000700252000c00e0000c0034008c08dd0066
:103a0000f00316000703de00868070000c00dd0066
:103a1000074bde00060070008c4cdd000743de0023
:103a2000868474000c44dd000c0252006120e10029
:103a300020003500610160000700280087816400d4
:103a4000f7ff270087836400070374000300e0008a
:103a50000600320082037300040032000000e80018
:103a6000e08048000188a3000e003a00f70f200014
:103a70000720e1004a003d000170a1004722dd005f
:103a8000810072008a8070000000be004f06be00f8
:103a90004f05be004f04be00000006006000b800e5
:103aa000faff37008100d1000080d3000402e80053
:103ab000eeff370004017800890174001b01070044
:103ac0008a807000f1ff370042010700070278008a
:103ad0000001fd008101fd003e0107008702780022
:103ae000850372000778a300040032000001fd0086
:103af0008101fd0051010700e4ff370085036200ea
:103b00000768a300080032000b50e10003003200f8
:103b1000f0ff2f00f1ff2700dcff37000001fd0060
:103b20008101fd00d9ff37000468a300d7ff3200f0
:103b3000faff3700f8ff2700888360000b003a0087
:103b40000000e00009003a008303640082837300f0
:103b5000020032000200be00ccff37000b50e10033
:103b6000ceff3a000200be00c8ff3700140020005c
:103b7000810064003eff3700f8ff27008883610062
:103b800004003a000200e00002003a008c007800d5
:103b9000beff3700150020008301640039ff3700a5
:103ba00001f827000000200081007500b7ff3700f2
:103bb000889fbe008a9fbe008c9fbe001b00200015
:103bc0000202be00058668000600280006066600a0
:103bd0004709de00f20fb200820032000243e80023
:103be00080003200c729de00f30fb2007d003200f2
:103bf0000343e8007b003200f107b2000170a0002f
:103c0000f507b2000570a000c708dd004903de001b
:103c1000868070004700dd00c72add004923de00f2
:103c2000868272004722dd00030551000403500024
:103c30008583580003003100000040008180480067
:103c40000a05e9008c1f78008a9fbe00040050001e
:103c5000858058000402420085824a00000040002e
:103c6000818048000005eb000004be006033b8000e
:103c70000406be000d48e1005600310011000900a5
:103c80004dccd8000c01b8000d02b8008481410071
:103c900060824a008283530003045c0084845c00d9
:103ca00060055d000a00e00025003a00800578000c
:103cb0000d40e100490031008800780007007800dd
:103cc000110009004d88d8000c01b8000d02b800a1
:103cd0008481410060824a006003110083835b009d
:103ce00004045c00e0845c000900e00021003a006c
:103cf0004f01be000300e0002b003200e301600032
:103d0000070673008c8171000100320064007000ae
:103d10004200de004e5edd000c007000c258de0086
:103d200001e0a000ce000700cf0178008180710083
:103d30004f06be004f05be004f04be000000060047
:103d40008c8343000d044c00e0844c0060054d0062
:103d50000000e9000a00e000d4ff32008c83430039
:103d60000d044c00e0844c0060054d000000e900ab
:103d7000ceff37000c0343008d834b0060044c00e2
:103d8000e0844c000000e9000900e000d8ff3200a8
:103d90000c0343008d834b0060044c00e0844c0016
:103da0000000e900d2ff37004200de004e5edd0079
:103db0000c007000c258de0001e0a000cf017800c6
:103dc0000300e000daff320060001000e08018001d
:103dd000d7ff3700f0ff2f00aaff3700f0ff2f00ba
:103de000b9ff37000404be007a0007008706780098
:103df0000004fd008104fd007600070007836600d3
:103e00000678a300030032000960a7000800be0086
:103e10002c0037000d78a300020032000800be001d
:103e2000280037000778a30026003a0001f0a1001f
:103e300009f0a1000668a30003003200f1ff27008b
:103e4000f0ff2f00baff37000d68a3000300320017
:103e50000800be008c807000b5ff37000768a30023
:103e600007003a000648a30003003200f1ff2700d4
:103e7000f0ff2f00aeff37000d48a3000300320013
:103e80006000b8008c807000a9ff37000748a300cd
:103e90000400320001f82700000020008c80700030
:103ea000a3ff3700c10007000004fd008104fd00ee
:103eb00002057800bd0007000802be008a017800f4
:103ec00059ff37000160a000120220004240880024
:103ed00097ff37000100e000120032000500e0000b
:103ee00010003200889fbe008a9fbe008c9fbe00db
:103ef0000006eb0001f8a300030032006000100090
:103f0000e08018000cf0a00005f8a30003003200c8
:103f100060021200e0821a000cf0a2008005eb00a3
:103f200041ff37006000b800020005000100e0001a
:103f300026003200610111007810e10023003c00ee
:103f40006022b8007010e1000400350080027800a3
:103f5000010078008000eb00700151000200e000d9
:103f60000900340070031100062add00822ade00f9
:103f70008603dd00878272000200de00860bdd0012
:103f8000070070008208de0084817100f4ff2700c2
:103f9000048262008481710004002800848262002f
:103fa0006102600005f0a6000000060004827100b6
:103fb000070032000000e800e08048000000060032
:103fc0000002be006000b800efff37006000b800dc
:103fd000000006002700200001f0a70017002000c5
:103fe000470bde00f60fb200040032000643e80083
:103ff0000a0032004702b300000006000103780007
:10400000f607b2000603700002003a000703b3008f
:10401000000006008702b3000000060001037800dc
:10402000f607b20006037000020032000770a0001d
:10403000000006000760a000000006000478a3004e
:10404000040032000578a300030032000168a300d9
:1040500001003a000200be000160a000000006005e
:1040600081017000270032008002eb0001f8a300fc
:104070000300320060001000e080180015002000ee
:10408000f40720000202420020003400f703200061
:10409000870360000604200000036300020820007c
:1040a000000161004700de00c909dd0000807100e9
:1040b000c708de000600e000080032008703710038
:1040c000060032001000b0000180b0000188a3009b
:1040d00002003200c108de000402e800f107b2006d
:1040e000f30f20000320e10003003d004722dd0024
:1040f000810072002900370001f827000000eb0062
:10410000260037006000b8000000060068021200b8
:104110007f20e100020034006000b8001f0037007b
:104120006011b8007020e1000400350080017800c3
:10413000010078008000eb00700252000400e000f3
:1041400009003400f00312000719dd008419de00b5
:104150000703dd00868171000400de00070bdd002f
:10416000060070008408de00f7ff270083836300e9
:104170008703710006002800030363000700320074
:104180000700e00003003a00610160000281730053
:10419000020032001000b0000180b0000500a6004f
:1041a0000000060001f0a000000006004f0ade003b
:1041b0004709de00f107b200f20fb2000b00320037
:1041c000f207b1000170a000c708dd00c901de00e0
:1041d000838070004700dd000400a6000000060098
:1041e00060001000e080180000000600810f7000e1
:1041f00001003a00000006008182cf000500e000c7
:1042000010003e008082cf00ee8242007028e10064
:104210000400390007003e00800078000000eb0039
:104220000e003700708312008600de000500dd00fe
:104230000a003700708352008600dd000000eb00aa
:1042400006003700e28252008508dd00708312000c
:104250000603de00868070000500dd007507b000f3
:104260000501ea000400a60000000600600010003e
:10427000e080180000000600881f78000304780022
:104280000300e00007003d0060001000e08018001f
:1042900060011900e081190002003b0001f02d00cf
:1042a000030037000400070008f0a70001f0a00099
:1042b0004f04780000000600889fbe008a9fbe0061
:1042c0000082700004027100048271002600320036
:1042d0000004be000200be006011b8006b0920009f
:1042e000950220000182cf000a0039000541b1008b
:1042f0000082cf00070039000541b1000982cf00dc
:10430000040039000541b1000882cf0001003900e6
:104310000541b10005425200120032000a003b0084
:1043200082817100610164008100d1000080d300ae
:104330008984d3000884d3008b05e8000442e80098
:10434000f7ff3a00070037000804440089844c0056
:1043500000004800818048008b05e9000442e90024
:10436000f9ff3a00030007004f05be004f04be00ee
:104370000000060081002000618055000b003d0018
:104380000b00200061fe2f000100e1001d00340041
:1043900082817100610164008904d1000884d30026
:1043a0000000e800faff3a0071002000610064009c
:1043b0000300700002006000090032006104440044
:1043c000e0844c000988a500050032008b05e80058
:1043d0006808e10002003a008904d1000884d30093
:1043e000f20f20000258e10005003d00c75ddd002e
:1043f000f907b20089807500080078000000060007
:104400000bf827008b007800000005000000fa0080
:1044100068815700cfb89700e00207000080fa00db
:104420000000060002000700e0023700000006005e
:104430004200fa00889fbe008a9fbe008c9fbe008b
:1044400020079800110f9800034f98001100780082
:10445000400f980091009000610f98009e09900015
:10446000a3019000330f98001e0a900044029000b0
:10447000140798009e0a9000b50290000527980046
:104480003204be002205be006022b8006033b800ce
:104490000800be000a01be00750607000000e0002b
:1044a00003003d000bf0a200d0c2b30004003700af
:1044b0004e0b90000628a30009003200b0c2b300e2
:1044c0008e239000804b78003e0890000000e900a9
:1044d000700f980011002000510f98001000370055
:1044e0004e0990000238a3000900320000c2b30058
:1044f0008e219000804978003e0a90000402e90075
:10450000740f980015002000550f98000400370024
:104510003e0b9000760f98008003eb00570f980039
:104520000800be000a01be00c0ff0700f4ff2f0014
:10453000f5ff2f00f6ff2f00f7ff270004026000b1
:104540008582600006036100878361006000b80017
:104550000200200003ff27000020e10001a8e10085
:1045600002b0e10003b8e10011003a000e489000eb
:104570008000fb001104b1000e219000de099000c4
:1045800003004100f98f500002003e0081872000a7
:1045900001003700c187200030050700c0872000d8
:1045a000350507005e0a9000040140001500370041
:1045b0000020e10001a8e10002b0e10003b8e10041
:1045c000130036008e4a90008500fb001104b100f4
:1045d0000e239000de0b900007004300f98f50007f
:1045e00002003e00018820000100370041882000c1
:1045f0001a050700408820001f050700de0890000c
:10460000010140004e0a9000be09900050023700a0
:104610006022b8006033b8000800be000a01be0086
:10462000130607000000e0006a0032006022b800b4
:104630000600200007ff2300441798005517980034
:1046400066179800771798008006eb000800be00f8
:104650000a01be00001f9800111f9800221f980039
:10466000331f98000e269000070037008d06e800e3
:104670000802be000a03be004417980055179800b0
:1046800066179800771798006022b800060020008f
:10469000470224004e109000de1090006e11900032
:1046a000fe119000620707000004be000205be0074
:1046b0000002be000203be000e1890009e1890007b
:1046c0002e199000be199000e90507000000e000d7
:1046d000e6ff3d000c2798000006eb004e1490000a
:1046e000de1490006e159000fe1590002500370036
:1046f00040ed2f00808f560019003d000c00e000b7
:1047000016003a006022b800060020000735240099
:104710000e1890009e1890002e199000be1990005f
:10472000430707000002be000203be00041f9800fa
:10473000151f9800261f9800371f98006022b800a8
:1047400006002000073524000800be000a01be0054
:10475000370707000004be000205be001c00200051
:104760006022b80006002000470224000800be00b6
:104770000a01be007f0607000004be000205be005d
:104780008d06e9000802be000a03be000e18900064
:104790009e1890002e199000be199000b4050700d5
:1047a0000000e000d2ff35000800be000a01be0094
:1047b00040179800511798006217980073179800d7
:1047c0000e1c90009e1c90002e1d9000be1d90009f
:1047d000080037006022b8000600200007ff230011
:1047e0004417980055179800661798007717980097
:1047f0008006eb008e4a90000500fb00b60407001f
:10480000104f98006e0b9000600020000600e00042
:10481000010035006e08900071c6b3009e4b9000f9
:1048200081cf53000a003a00ee0890000100e0003a
:10483000cf013200cf0137008d0f5000d3013c0073
:10484000001f980052c6b300425f98001e00370058
:104850009e499000435f98000200370064c6b30091
:10486000445f98000000e800001f980060c6b30095
:10487000ce5a900080cf520013003a000d00e000a5
:1048800008003d006000b8000200200003ff230084
:1048900040179800511798006217980073179800f6
:1048a0008006eb0061c6b300415f980070c6b3009c
:1048b0001e499000804f5100030032008e19900075
:1048c0008d814100031f98004e129000de1290006f
:1048d0006e139000fe139000441f9800551f98001f
:1048e000661f9800771f98000800be000a01be00ee
:1048f0000017980011179800221798003317980096
:104900000006eb000802be000a03be005407980030
:104910006507980076079800070f98003100370068
:104920004e1a9000de1a90006e1b9000fe1b900045
:104930000e1090009e1090002e119000be1190005d
:104940000c060700640807000004be000205be0054
:104950007005070080027800250f98004e1a90001d
:10496000de1a90006e1b9000fe1b90000800be0037
:104970000a01be00ae0607000e1290009e129000c3
:104980002e139000be139000a90507000002be0080
:104990000203be0007f0a200041798001517980044
:1049a00026179800371798006022b80006002000ec
:1049b000470224004e189000de1890006e199000f7
:1049c000fe199000eb0507000002be000203be00c6
:1049d000441f9800551f9800661f9800771f980085
:1049e0000c06e8008e1a9000850f5600ccff3500ab
:1049f0005e049000ee0490007e0590008e0d900005
:104a00006022b80006002000470124004e189000e4
:104a1000de1890006e199000fe19900084060700c1
:104a20000002be000203be00441f9800551f9800fc
:104a3000661f9800771f98000e1090009e1090003f
:104a40002e119000be119000090507000000e00043
:104a50000f0035004e1a9000de1a90006e1b900079
:104a6000fe1b90000e1090009e1090002e119000e2
:104a7000be119000fe0407000000e00011003a00a3
:104a8000ae0a90000508a300080032000d003700b0
:104a90006000b8006011b800401f9800511f9800d6
:104aa000621f9800731f9800060037006022b8004c
:104ab0006033b800441f9800551f9800661f980087
:104ac000771f98004e1a9000de1a90006e1b90001f
:104ad000fe1b90000800be000a01be005a05070038
:104ae0000002be000203be000417980015179800cc
:104af00026179800371798006022b800060020009b
:104b0000470224004e109000de1090006e119000bd
:104b1000fe119000460607000004be000205be001c
:104b20000002be000203be000e1090009e10900016
:104b30002e119000be119000d20407000000e0008a
:104b4000090035008d06e80060c6b300ce5a90001b
:104b500080cf520008003a000e1b90000603e800c8
:104b6000061f9800110037004e149000de149000cc
:104b70006e159000fe15900050c6b3004e5990007f
:104b8000804f510009003a000802be000a03be002f
:104b9000441f9800551f9800661f9800771f9800c3
:104ba0008002eb0045179800070037000800be00a0
:104bb0000a01be00401f9800511f9800621f980014
:104bc000731f98004d1798005e0e90000001eb00d7
:104bd000220f980032079800520798000d0f7800b6
:104be0006a0037004e1a9000de1a90006e1b90008b
:104bf000fe1b90000e1090009e1090002e11900051
:104c0000be1190005b050700b30707000004be005b
:104c10000205be00bf040700e90f50000100340088
:104c200090002000ce0990000348a3000c003a0039
:104c30000000e0000a003a0071c6b3001e4a90006e
:104c4000814f520006003a00ce1290000500e000ad
:104c500003003d002e0b90008606e800230037007d
:104c6000be0390000700e0000c003a00ce10900058
:104c70000100e00009003d00e1c2b3000e219000f8
:104c800001717e000c06e800fe0990008301e90036
:104c9000730f980014002000340798008e229000b3
:104ca0000c814200ae0e90008501780003003700b1
:104cb00001c3b300015978008d06e9000d00e00042
:104cc000fbff3a00032798002e0b900006064600d3
:104cd0000043b00080717e000c06e8000680ea0008
:104ce000fe0b900080834300770f98004e1a9000cf
:104cf000de1a90006e1b9000fe1b90000800be00a4
:104d00000a01be00ca0507000e1290009e12900014
:104d10002e139000be139000c50407000002be00d1
:104d20000203be0007f0a2000417980015179800b0
:104d300026179800371798006022b8000600200058
:104d4000470224004e189000de1890006e19900063
:104d5000fe199000070507000002be000203be0016
:104d6000441f9800551f9800661f9800771f9800f1
:104d7000ce1290008502e900451798005e0390006e
:104d80000603e800560798002d0f9800de039000f8
:104d90000e189000808f530005003d009e08900083
:104da0004100900065005000800f56008dff3900d3
:104db0009e0678003e0190000200e00007003a00e5
:104dc000ce0990000348a30004003200e0c2b30003
:104dd0000e22900000727e000c06e8008e229000e9
:104de0000c8042000048eb0051c6b3004e5b9000bf
:104df000814f530038003a009e0390008700e9007d
:104e00000041eb0082f278008001eb000d00e00031
:104e100002003d008d06ea00130020002200200061
:104e200001037800fe0a90008e23900000047800b1
:104e30000a00370001037800a400200011000900d7
:104e40008406d80001027800800678000443b00090
:104e500084737b000201e9008502e9008600e90015
:104e60000d00e000f3ff3a000200e000f1ff3c001b
:104e7000750f98000727980008007800018243000a
:104e8000b2c2b3000300e00001003200d2c2b3009e
:104e9000024a78000101e9008e21900082804100e1
:104ea0008e4a90000502fb001404b10053c6b30003
:104eb000f90f520001003e0053c4b300834878004c
:104ec0007e0b90000683e900760f9800820f560053
:104ed00001003d00e1020700ce0b900063806300fb
:104ee000e20f500015003a007e0890000000e0003c
:104ef000120034000e209000df0207008e21900087
:104f0000040037007e09900082804100e370780041
:104f10000000e900de0a9000850f5000f9ff3d0017
:104f200003279800058041007e09900001032000be
:104f3000660207000003eb00360f98000e20900079
:104f4000cd0207004e0a9000be09900000017800d3
:104f50008e2090002e009000460007004f06be00f5
:104f60004f05be004f04be000080fa00000006009e
:104f700010002000e48f46002ffe3d00001f980027
:104f800057c6b300475f98004ffe37000d00e000a2
:104f900032fe3500001f980042fe37008201780083
:104fa00001017800f1ff2700d2023700881f780046
:104fb0000004780000082000808f500017003500a2
:104fc00010082000808f50000b00340030082000b3
:104fd000808f500011003a009200780068805000e5
:104fe000000978003002be002003be00049cbe0011
:104ff0000694be00070037009202780064805200d9
:10500000000978001000be00a3030700009cbe004a
:105010000294be0010002000010037000000eb00e9
:105020004f04780000000600889fbe00000478004e
:105030004800900082047800808f54000100360000
:1050400080047800090178005800900018020700d9
:10505000580090000900400050049800c8009000db
:1050600089845000490498000048eb004f04be00ba
:1050700000000600f2874700889fbe008a9fbe009e
:105080008c9fbe008e1f7800800478000105780098
:1050900002047800830578006107620002003a008c
:1050a0008b0f540008003900080178008a0078004e
:1050b00009007800dcff07008b0f54000200390064
:1050c000880578001e003700088655000c0178001e
:1050d000f00f5600010036000201200001022000fe
:1050e0007e805700f90107008c0678000500370024
:1050f00002012000fe80570009007800caff070067
:10510000f0865600ef8f5600f9ff3e004461de0046
:1051100000ff2f000091b90002014600fe805700f9
:1051200009007800c0ff07000e00e00004003a000c
:10513000080178008a00780009007800baff0700ab
:105140000b0078004f0778004f06be004f05be00e9
:105150004f04be002f01b100000006000000050052
:105160000000050000000500000178000040eb0091
:105170008080fb00818040002386200063c278008d
:105180000404e00003003a003086200060c078008c
:105190000000060092017800934f520004003a008c
:1051a0003086200060c078000309e8000100370065
:1051b0000040e800ea4f5000edff36000000060016
:1051c000f6874700889fbe008a9fbe008c9fbe0066
:1051d0008e1f7800000578000104780083057800b0
:1051e000040678000000eb00c0b79f008080eb0051
:1051f000d1b79f00e0b79f00f2b79f0000082000e2
:1052000080bf9f0098007800010078008004eb00c8
:10521000010037008904e800304178000204e00012
:105220000300320053c2b300834f5100f9ff3a002c
:105230000900e00004003200090178000a0078004b
:1052400079ff0700188c44001807780050c2b3009b
:105250009e4f10003f013a000e07e8000e0c780048
:1052600010003700cfb097000100a0000b003700fe
:10527000cfb097000110a00008003700cfb0970012
:105280000120a00005003700cfb097000130a0003a
:1052900002003700cfb097000140a000c1b79f00c7
:1052a000000ce8001800780090407800b2c2b3000b
:1052b00082cf5000f1ff320007003c0002c2b30071
:1052c00082cf5000f0ff320032c2b30082cf5000d4
:1052d00007003a00efff3700d2c2b30082cf500080
:1052e000e0ff320002c3b30082cf5000e0ff320083
:1052f000a2c2b30082cf50000d003a00000ce800bb
:105300001c80e900000e780010007800e0b79f00d4
:105310000000e0000f003d00cfb097000100a200a8
:10532000c1b79f000000ea00e0b79f000900370006
:1053300039010700e0b79f0001003700000ce800ca
:10534000180078009000fb000103b100e98f5000c5
:10535000faff36004fb097000008a30002003200a9
:105360000010a100c0b79f0018007800e1c2b30090
:1053700090cf100016003a008000eb00d1b79f00dc
:105380000000e800000c7800a1c2b30090cf10002c
:1053900006003a00000ce8001c80e900000e7800ce
:1053a00010007800d0b79f00090037001a010700ed
:1053b000d0b79f0001003700000ce800180078000b
:1053c0009000fb000103b100e98f5000faff3600a6
:1053d0000800780064ff0700804678001800780015
:1053e0001000fb00bc01070091062000810f500057
:1053f0003800320012003c0041062000810f5000ae
:10540000340032000a003c0011062000810f5000d9
:105410002000320031062000810f5000a000320031
:1054200051022000810f5000bc003a00b400370048
:1054300071062000810f5000b8003c008800370042
:1054400001072000810f50005c00320007003c0083
:10545000e1062000810f50007a003200f1062000a2
:10546000810f5000ad003a0039003700510720008d
:10547000810f50002700320081072000810f50006b
:105480004200320031072000810f5000a3003a0093
:105490008f0037008d80fb000c01780000fe2f008c
:1054a0000f004000c1fe07000000e000a80032002d
:1054b00018007800000ce8009041780002fe2f00f0
:1054c0000f014100f88057000a00780024ff070010
:1054d0000e0037008d80fb008c0178001200200048
:1054e00000fe2f000f004000a70107000000e000b1
:1054f00097003200180ce80002fe2f000f01410057
:10550000f88057000a00780014ff070080844400e8
:10551000900037008d80fb008c0178000001eb00cb
:1055200000fe2f000f004000970107000000e00080
:1055300087003200180ce80002fe2f000f01410026
:10554000f88057000a00780004ff0700efff3700db
:105550008d80fb008c0178000001eb0000fe2f0025
:105560000f004000880107000000e00078003200d2
:10557000180ce80002fe2f000f014100f8805700d0
:105580000a007800f5fe0700e0ff37008d80fb0081
:105590008c0178000001eb0000fe2f000f0040009e
:1055a000790107000000e00069003200180078006f
:1055b000000ce800904178001c0037008c01780056
:1055c0000001eb00010f200000fe2f000f00400043
:1055d0006d0107000000e0005d003200180ce800db
:1055e0000fb097009fb097002fb19700bfb1970001
:1055f000e00f5000e08f5800e00f5900e08f590095
:1056000009003a00cfb597006fb49700a08520003d
:10561000190107000b02780088017800000178006a
:10562000a18520004700370083c7b30002fe2f008a
:105630000f014100f88057000a007800c8fe0700fb
:10564000b2ff37000b8144008d80fb008c01780095
:1056500000fe2f000f0040009f0107003c003700b4
:105660008d80fb000c01780000fe2f000f00400031
:105670004efe07000000e000350032001800780000
:10568000000ce8009041780002fe2f000f0141005d
:10569000f88057000a00780065fb07009bff370081
:1056a00000c8b30080cf560029003a00180ce8006b
:1056b0001c80e900000e780010407800e0df9f00b9
:1056c00013002000e2fd2f000f0141000800370009
:1056d00000c8b30080cf56001d003a00180ce80047
:1056e0001c80e900000e78008001eb0010017800ba
:1056f000f88057000a0078009afe070083ff370001
:1057000000c8b30080cf560011003a00180ce80022
:105710004fb29700efb19700080037000e0c7800e9
:105720000000eb00c0b79f00e0b79f000080eb00d7
:10573000d0b79f000002eb00840178001200200027
:10574000018620000a0078004afe07006fff37003c
:10575000180ce800090078004f0778004f06be00db
:105760004f05be004f04be006f01b10000000600ef
:105770008200fa00889fbe008a1f7800000578002a
:1057800082047800c13f9f000004eb001000370046
:105790000902780088017800a2f72f000f0141006c
:1057a00081f72f008f8040000a00780084fe0700f8
:1057b00008004000880f500004003d00b0042000a5
:1057c000404488000084eb000400370000047800a7
:1057d0004f3897001004e000edff3a000800780011
:1057e0004f0578004f04be000080fa00000006005c
:1057f000800078001000200002022000828f5000fc
:1058000004003200e9805000e48f500001003600af
:105810000000eb0000000600889fbe008a1f780091
:10582000000578000a047800984478000805e8002c
:105830000900fb00eeff07000000e000f9ff3a005e
:10584000b0c2b30080cf540005003200d0c2b30014
:105850008000eb0080cf540005003a0002003700c2
:105860008000eb0001003700110020000804e80070
:105870000000eb00030037006a02b900020052008a
:105880000003b0003801fb0003fd2f0082814100be
:10589000e98f5100f8ff36000100e00001003a00f6
:1058a0000000ea004f0578004f04be00000006002b
:1058b0008001780002003700b15978000201e90048
:1058c0000200e000fcff3a0000000600889fbe00d6
:1058d0008a9fbe00800478000200e0005b00320076
:1058e00001407800814c780082814400f1f99f00ea
:1058f000e20f51005500360091449800a1449800f1
:10590000e1f99f00d1f99f00e60f51004f003600ea
:10591000b1449800c1f99f00e80f51004b003600d8
:105920000905ea00630565000a8444000a05510080
:10593000c1ff2f00010565000080fb008000eb0027
:105940001210200013102000b3010700008cbe00cd
:105950000a01440060b99f0071b99f00e80f55002b
:105960003a00360020049800310498004004980062
:105970005104980020b99f0031b99f0040b99f00a1
:1059800051b99f00f80f55003000360060049800b0
:1059900071049800000c9800110c9800200c9800dd
:1059a000310c9800400c9800510c980020b19f00d9
:1059b00031b19f0040b19f0051b19f0060b19f0085
:1059c00071b19f0000b99f0011b99f00640164008c
:1059d0007801410002044400020555006011b8003e
:1059e0000203be000002be000403be006022b80035
:1059f00000007200818072000201730083817300d5
:105a000010003700009cbe000294be0040049800c5
:105a1000510498006204980073049800000c9800e8
:105a2000110c9800220c9800330c9800400c980040
:105a3000510c9800620c9800730c98000a02b10097
:105a40000802b000ff0f5500eeff3e00090078008d
:105a50004f05be004f04be0000000600881f7800fe
:105a60000004780008007800d300070008007800e0
:105a70004f04780000000600800078000400370022
:105a80003104e00002003a0000005100000006006e
:105a9000010178000108a300f9ff3a0081017800b4
:105aa00031017800f4ef2f00020242000281ea0087
:105ab000020162000408280004016100f7ff3200bf
:105ac00083007800010178003104e000fdff3a0016
:105ad0000000510000000600f1fb2f008080400014
:105ae000f98f500001003e000050a00000000600a9
:105af000f9ff3700f28747008e1f78000202780016
:105b0000030178000000e000020032000007780086
:105b100001003700728757008002eb000100e000af
:105b2000010032008102e900708057000600090080
:105b30000018eb000080eb0080bf9f0023102000c6
:105b400093bf9f00aebf9f00b1bf9f00c5bf9f0026
:105b50000100e00003003d00b10420004144880042
:105b600006003700004feb00eebf9f00debf9f0036
:105b70008400780070805700af0007004f0778005e
:105b80002f01b1000000060084082000848f50001f
:105b90001d0032000d003c0014082000848f5000ce
:105ba0002700320002003c000408200004003700f7
:105bb00024082000848f5000340032004408200064
:105bc000848f500043003a0036003700040a20005a
:105bd000848f50002700320004003c00040920009c
:105be000848f50003b003a0028003700020c200050
:105bf000828f50002f003200020f2000828f500051
:105c000034003a002b0037009380e9000200e000e6
:105c100005003200810978001102fb00cfa2de00ee
:105c2000612bb90028003700810978001142780003
:105c30000482fb008002eb006033b80022003700d2
:105c400013027800e40052000200e0000500320078
:105c5000810978001102be004fabde008603780098
:105c600019003700810978001102be006033b800c6
:105c7000150037009380e90081097800110278004f
:105c8000cfa2de00612bb9000f003700930278002d
:105c9000e8805200810978003102be002103be0075
:105ca000090037009380e9000200e00002003200a2
:105cb000f1ff37009380e900810978001102780034
:105cc0008002eb006033b8000498be000690be006e
:105cd000100005000000050044082000848f5000db
:105ce0002500320008003c0014082000848f50007a
:105cf0001400320024082000848f50002400320059
:105d0000040820000c00370004092000848f500094
:105d10001f00320004003c0084082000848f5000e3
:105d200024003a000e003700040a2000848f50003f
:105d300011003200040c2000848f50001d003a0036
:105d40000d0037009380e900810978009100780008
:105d500001087800cf91de008288be001400370071
:105d60009380e900810978009100780001087800ab
:105d7000824878000e0037009380e900810978009e
:105d80009100780001087800820878000800370048
:105d90009380e9008109780091007800010878007b
:105da0006112b900612bb9008498be008690be00d4
:105db0001000050000000500010178008001780056
:105dc000008268000408a3000500320013003700b9
:105dd00032407800805978000004e000140032005e
:105de000030278000208a300f9ff3a0003007800dc
:105df000010037000318780082007800b2017800b3
:105e0000f5ef2f00838242000382ea0004826200e1
:105e10000508280005026200f6ff32000002780043
:105e200031417800025878000204e000fbff3a009c
:105e300004007800000006000200fa00881f7800c5
:105e400000047800e2bf9f006481570008007800da
:105e500047fe0700980090000148a30001003200af
:105e60000080eb004f0478000080fa00000006007c
:105e70008f1fd1008f0207008f87e9000000e0002c
:105e800000000600809feb008a0207008f87e90070
:105e90000000e000000006008103780049000700d0
:105ea0000001be006000b8000478a30013003a00af
:105eb0006220e10015003e000d0039008301d10091
:105ec0000281d3008180d3008301d1000281d300fd
:105ed0008180d3008301d1000281d3008180d3006f
:105ee0000538b000c42add00f300b20083817200df
:105ef00007f0a70003f0a0000000060083ff2700c2
:105f0000020020006110b900f9ff370003ff2700ed
:105f1000f7ff37001400fa00889fbe008a9fbe007a
:105f20008c9fbe000004be000205be006800470052
:105f30000a90be000890be00990207000070a700fa
:105f40000bf0a100304320009e029000808252009e
:105f5000b0fe2f000028e10011003d00b0fc2f0032
:105f60000028e100150034001e0990008e08900002
:105f70007e0090000501b0000201d1008180d300b5
:105f80000080d3008502e800fbff3a000b00e00030
:105f9000be023b0060001000e0801800bb0237002a
:105fa000f0ff2f00f1ff27000b00e000b7023b00dd
:105fb0000100280000002000b40237006000b80093
:105fc000b2023700c70ade00f107b200f50fb200d7
:105fd00008003200e1cf4200020032000170a00050
:105fe00024000500810f7000010032000408050044
:105ff00044000500810f700002003a001400050003
:106000008502e9000000400081c04800fcff3b0021
:106010000170a00024000500020ab900001bb900ad
:106020000200b80081004200810043000000060029
:106030008c9fbe008a9fbe00889fbe00ca010700d9
:106040000bf0a200040037008c9fbe008a9fbe00a8
:10605000889fbe00c40107000c48e1000b003a0015
:106060000c40e100020032008b01070040003700c5
:106070008b066d003e0032000af0a100f301200003
:10608000f2ff2f006110b900390037000c40e10029
:10609000370032000940e100010036007e010700b0
:1060a0008a856d00cf5dde000b0575000006eb00f4
:1060b0008804fd0089045400010032007d010700be
:1060c0000a04e00011003a000800e0002800320055
:1060d000040040008580480006014900878149008e
:1060e0000358a300180032008301d1000281d300bd
:1060f0008180d3000080d3000c86d30001003900da
:10610000610676000804e80018003700040050001b
:10611000858058000601590087815900060031002a
:106120000af0a2000c06ea0060001800e0801800e7
:1061300060011900e081190003003a000004eb003f
:106140000005eb000a0037000348a30007003a00ef
:106150000c0646000000480081804800020149000a
:10616000838149000804e900f7ff3700af013700d9
:10617000c90137008c9fbe008a9fbe00889fbe0069
:10618000790107000b056d000940e1000a003a00a3
:106190000800e000020032000c40e10006003a0076
:1061a0000af0a1000c047800f3012000f2ff2f0098
:1061b0006110b9009d0037000c40e1009b003200e7
:1061c0000800e000990032000c48e10002003a00ab
:1061d0000004eb00030037000900e00004003a006f
:1061e0000c0478006000b8006011b8008f00370020
:1061f0000348a30006003a000000400081804800e8
:1062000002014900838149000804e900f8ff3700d2
:106210000748a30006003a000402420085824a00b3
:1062200006034b0087834b008904e900f8ff370021
:10623000fd3f20008d845400090454008a1f78001b
:10624000881f780000047800810478000205780037
:10625000830578006000b8006011b8000d042000cc
:10626000050037000804440089844c000a054d00ed
:106270008b854d00080031000404540085845c00c7
:1062800006055d0087855d008381d2008d06d30001
:10629000f4ff3b00070037000404440085844c00f1
:1062a00006054d0087854d008381d2008d06d30001
:1062b000ecff3b000804440089844c000a054d00b3
:1062c0008b854d00080031000404540085845c0077
:1062d00006055d0087855d000281d2008d06d30032
:1062e000f4ff3b00070037000404440085844c00a1
:1062f00006054d0087854d000281d2008d06d30032
:10630000ecff3b000804440089844c000a054d0062
:106310008b854d00080031000404540085845c0026
:1063200006055d0087855d008180d2008d06d30063
:10633000f4ff3b00070037000404440085844c0050
:1063400006054d0087854d008180d2008d06d30063
:10635000ecff3b000804440089844c000a054d0012
:106360008b854d00080031000404540085845c00d6
:1063700006055d0087855d000080d2008d06d30094
:10638000f4ff3b00070037000404440085844c0000
:1063900006054d0087854d000080d2008d06d30094
:1063a000ecff3b000b00e00004003d00040444004f
:1063b00085844c0006054d0087854d000006eb00e6
:1063c0008301d1000281d3008180d3000080d300fb
:1063d0000c86d3008301d1000281d3008180d300d9
:1063e0000080d3000c86d300890474008b057500ef
:1063f0008b84740001003200610676004f0478003f
:106400004f0578000348a30007003a000c06460039
:106410000000480081804800020149008381490052
:106420000804e900f7ff3700000137001a013700c0
:106430008c9fbe008a9fbe00889fbe00ca000700d6
:106440000b056d008a0578000c40e10008003a0059
:106450000900e00082003a000af0a1000c04780074
:10646000f3012000f2ff2f006110b9007c0037001b
:106470000c48e10004003a00870007000900e00032
:1064800077003a00f4ff37000800e00074003200a3
:106490000900e00002003a007f00070070003700aa
:1064a000ed3f20008d845400090444008a1f7800c9
:1064b000881f7800871f7800861f7800851f780066
:1064c000841f7800cb19dd00c515de008b857100b7
:1064d0004b11dd00450dde000a057100cb08dd0023
:1064e000c504de00898470004b04dd000440b80060
:1064f0000546b8008c80400060814e00044eb80014
:106500008c8040000d0149008001eb000318ad00b4
:106510000456b8000c0141008d8149000002eb00d7
:106520000420ad000646b8000c0141008d814900f1
:1065300060024a00054eb8000c0141008d814900ff
:1065400060024a000556b8008c8141000d024a00e5
:106550008002eb000528ad000746b8008c814100a1
:106560000d024a00e0824a00064eb8008c814100cc
:106570000d024a00e0824a004f0678000c5eb80027
:106580008c8141000d024a00e0824a000656b800a4
:106590000c0242008d824a000003eb000630ad0081
:1065a000074eb8000c0242008d824a0060034b0087
:1065b0004f0678000c5eb8000c0242008d824a0043
:1065c00060034b000756b8008c8242000d034b005d
:1065d0008003eb000738ad004f0678000c5eb80072
:1065e0008c8242000d034b00e0834b004f06780085
:1065f0000c5eb8000c0343008d834b004f04780001
:106600004f0578000748a3000a003a000000400048
:1066100081804800020149008381490004024a0048
:1066200085824a0006034b0087834b000804e9007b
:10663000f4ff3700030678008080700082807000cd
:1066400001003200610676008701780006017800bb
:10665000850078000400780088047800780037000e
:106660008d0037008c06460002003a000000a600ac
:106670000000060060004800e0804800600149001a
:10668000e08149000350a600000006008301d1000c
:106690000804e800000006000002fd008102fd0081
:1066a0000203fd008303fd008804fd008a05fd0050
:1066b000000006007048e1001a0039007d03200048
:1066c0000d48e1000a003900810570008306710061
:1066d0008c8575008d8575000006eb000cd8e700f1
:1066e000610676006000b8006011b8000000060086
:1066f0007048e1000b0039008c0578000006780036
:106700000100780082007800030178008001eb002e
:1067100003d8e70061067600f0845400f4ff3a00e5
:10672000000006006160e1000c48ad00f085140037
:106730008b06dd000966de000d0676008b0edd009f
:106740000900de000d0070008b16dd008908de00f8
:106750008d8070008b1edd000911de000d017100bf
:106760008919de00000006000d002800fc7f2000d3
:106770000d856100441cde00ef8161000c046400a3
:10678000010032000340a0008d856300c43cde00a0
:10679000ef8363008c846400010032000740a00096
:1067a0000c40e10006003a00ef8661008286760028
:1067b000818676008086760001003200180037005e
:1067c0000c48e10007003a00ef86630086867600f9
:1067d000858676008486760002003200aeff0700d0
:1067e0000f0037000348a30005003a00810670003f
:1067f0008286760083867600010032000804e80075
:106800000748a30005003a008506720086867600d8
:1068100087867600010032008904e8000000060047
:10682000cf047800cf0578001b0037000002780005
:1068300081027800020378008303780088047800de
:106840000cf0a70087ff0700fd7f20000d40e1004e
:10685000040035000d0478006000b8006011b80035
:106860000d0037000800e0000b003c000400780039
:10687000850078000601780087017800e184140023
:106880008cff07000cf0a70076ff07000004eb0068
:106890000340a7000804e8004444dd006fc5610020
:1068a000880175004f04be004f05be004f06be00b4
:1068b00000000600889fbe008a9fbe008c9fbe001d
:1068c0000404be000605be00809fbe00829fbe007d
:1068d00021000700040678000800be000a01be007f
:1068e0001d000700840678004f03be004f02be0063
:1068f0008d4f76007fb0970013003300f0ff2f001c
:106900008b8f6b0006003b000d0666000c00a70095
:106910000a00370007f0a600100020000a00370028
:10692000880f5200898f5a008a0f5b008b8f5b00a3
:10693000030039001000200001003e00000020008c
:1069400007f0a7000000ea004f06be004f05be009a
:106950004f04be000000060005ff2700058261000d
:10696000070032000428e100010032002400050085
:106970000600070001003a00440005000408050075
:1069800002000700f9ff3a00140005006f82610061
:10699000810270008502710085027200000006000d
:1069a000800078005002be005003be004439de0073
:1069b000f700b200f37f20000301610009003200fc
:1069c0000218e10016003a0085017200830173008d
:1069d000838173000008200015003a004000200069
:1069e00013003700850172008301730083817300f7
:1069f00005003a0004a8be0006a8be001000200052
:106a00000b0037000201e9000402420085824a00bf
:106a100006034b0087834b000748a300f9ff3200b1
:106a20000740a00004a8be0006a8be002000200069
:106a3000800098009200980000000600680447005b
:106a40000294be000094be00fc0447008694be0081
:106a50008494be0009007800d1ff07000800780088
:106a6000cfff070099007800814f70000b003b00ba
:106a70000800be000a0007004f00b1000300370005
:106a8000f3ff2700f2ff2f006110b9004f06be0090
:106a90004f05be004f04be000080fa000000060053
:106aa000e48240001078a300070032006402400036
:106ab0001178a3003400be001401be0004003200af
:106ac0000330a700000006003500be001501be001f
:106ad0000330a000000006001800fa00889fbe00e6
:106ae0008a9fbe008c1f78000004be000205be0015
:106af0000802be000a03be00443ade00f07f200018
:106b00000006620020432000800f560067003c0012
:106b10006022b8006033b8000800be00d4fc070053
:106b20000000e000610032000802be000a03be005f
:106b3000b4b79f00c5b79f00d6b79f00e7b79f00c7
:106b4000e00f5200e08f5a00e00f5b00e08f5b0027
:106b50000b003d006022b80006002000073324002f
:106b60000800be000a01be0031fd07006022b80027
:106b7000060020000733240033fd07000a00370019
:106b80006022b80006002000073324000800be0081
:106b90000a01be002cfd07006022b800060020009c
:106ba0000733240022fd07000802be000a03be00ce
:106bb0001ffd07000002be000203be00f4b79f00e5
:106bc00085bf9f0096bf9f00a7bf9f00e03f2000aa
:106bd000800f560017003c007fb097008fb89700d9
:106be0001fb99700afb99700f0af9f0081b79f0022
:106bf00092b79f00a3b79f006044b8006055b800eb
:106c00003fb29700cfb297005fb39700efb3970002
:106c1000e00f5200e08f5a00e00f5b00e08f5b0056
:106c200022003d006044b8000a0020000bff2b004a
:106c30001e0037006022b8006033b8007fb09700b4
:106c40008fb897001fb99700afb997008dfc070068
:106c50000000e0000c0034007fb297008fba97006c
:106c60001fbb9700afbb97000800be000a01be0023
:106c7000f5fc07006022b8000600200007ff230093
:106c8000ebfc0700070037007fb297008fba970030
:106c90001fbb9700afbb97000800be000a01be00f3
:106ca000e9fc07000004be000205be000800be00ab
:106cb0000a01be004f0678004f05be004f04be001b
:086cc0000080fa00000006004c
:020000040000fa
:106cc800020400000e0100000f1100000f00000078
:106cd800020400000e1100001f1000000e0000004a
:106ce800020400000c040000040400000e00000070
:106cf800020400000e110000111100000e00000037
:106d08000204000011110000111300000d00000022
:106d18000a00000011110000111300000d0000000e
:106d2800050a000011110000111300000d000000f9
:106d3800050a00000e110000111100000e000000ed
:106d48004454000048310000312000005445000040
:106d5800535a000054000000445400004831000019
:106d68003120000045520000524f0000520a000036
:106d78000043000048450000434b00005355000005
:106d88004d000000544900004d4500004f550000db
:106d980054000000546500006d7000003a200000a7
:106da800252e000031660000b0430000200a0000d4
:106db800487500006d3a0000202500002e310000c3
:0c6dc800662500002520000000000000ef
:020000040000fa
:106dd4000a00fa00889fbe000040eb00004f7800d4
:106de400050037001e80fb00000047008040eb00d8
:106df400414098001e4fe8001e407800e44f5000c8
:106e0400f8ff36000000280090088800d802a90086
:106e1400da02a9000050260041002000f601070014
:106e2400da02a8000028200001002000f201070077
:106e3400d802a8000a21ef0006003700510880009c
:106e440000e82300808f500002003600e0ff2f008e
:106e540073003700d0168000610060000000e0007d
:106e6400f6ff32000a21ef000600370051088000c7
:106e740000e82300808f500002003600e0ff2f005e
:106e840067003700d0168000610060000000e00059
:106e9400f6ff3a000040eb00004f78002f00370067
:106ea4000a21ef00060037005108800000e82300a3
:106eb400808f500002003600e0ff2f00580037009a
:106ec400d0168000610060000000e000f6ff320090
:106ed4000a21ef00060037005108800000e8230073
:106ee400808f500002003600e0ff2f004c00370076
:106ef400d0168000610060000000e000f6ff3a0058
:106f04005108800000322000808f500012003600ab
:106f14001e80fb004300de00004078000081fb007f
:106f24000080fb0000004700404090008040780053
:106f34001e80fb000080ea00670060001300200050
:106f44000018dd000040780000c070008040780028
:106f540002004700414098001e4fe80070c2b30091
:106f64009e40780080cf5000cdff36004e40900008
:106f74000080fb008000eb001cf20700204088002a
:106f8400314088006e4090000080fb00cf80de001e
:106f940013f207000004be007e4090000080fb0056
:106fa400cf80de000ef2070002002000031224004e
:106fb400fef207000001be000800be0016f2070042
:106fc40000408800114088004e4090008080fb0003
:106fd4005e4090000080fb00808040006e40900086
:106fe4000080fb00808040007e4090000080fb0019
:106ff40080804000f00f200000806000100798009f
:107004000e4890008080fb001e009000808f50008e
:10701400020032000080eb00010037000000eb00aa
:107024004f04be000080fa00000006000200fa00cf
:10703400213a8000f0f32f0000806000203a88009d
:107044000100370000000000113a80000002200017
:10705400008060000000e000faff320040a7a900b1
:10706400f0c2a900f0e2a900f102a900f122a900ee
:10707400d9e2a900e882a900e8a2a900d022a800c8
:10708400d062a800e102a800e122a80039000700ac
:1070940020010700406a2b008f00070000602300d6
:1070a400e11620005401070049ff0700000f780093
:1070b4001e0078000000e000100032008040eb0069
:1070c40010c0b3004d000700006b2b0082000700c6
:1070d4001e007800e10f400002003a00d06b2b0044
:1070e4007d0007001e007800e20f400013003a0004
:1070f400606c2b0078000700100037008040eb0024
:1071040020c0b3003d0007002240800033408000cf
:107114000040800011408000829fbe00809fbe001e
:10712400e06c2b00801f7800a0802000b6f40700dc
:10713400ea875700a080200067000700e01680005f
:107144000080ea004f00de00004078000080fb0071
:107154004f00dd00e116800001f0a1000100700085
:10716400e016880000602300e116200022010700d9
:10717400cdff37000000fa000117800000f02f0057
:107184000080600000178800f002a900f022a90026
:10719400e822a900f402a900f422a900ec22a90023
:1071a40000502300c1002000130107008040eb00c1
:1071b40080c3b300110007008040eb0080c0b3001f
:1071c4000e0007008040eb0010c0b3000b00070066
:1071d4008040eb0060c0b300080007008040eb0073
:1071e400c0c0b3000500070000b82b000100200058
:1071f400010107000080fa00000006000400fa0004
:10720400204798003147980001178000f00f2000b4
:107214000100700000178800f422a800f402a900fd
:107224002117800000f02f000080600020178800e4
:10723400ec22a80000000000000000000000000094
:10724400101780004700de0061406000004f7800a6
:10725400ec22a9001e4078000004e000f4ff3a008c
:107264000117800000f02f000080600000178800e4
:10727400f422a9003e4090000080fb000000ea00d8
:107284004f00de00004078000080fb0061006000d9
:10729400a11780000100a10001007000a017880060
:1072a4002117800000f02f00808060002e409000a5
:1072b4000080fb000100700020178800ec22a80069
:1072c400000000000000000000000000ec22a90003
:1072d4000080fa00000006000400fa00100798007d
:1072e400860037001e009000104f78001e00fb003f
:1072f4006101b900000520000100200002004000e7
:1073040083804800c204200003002000820f500044
:10731400838f58006c003e00006001006700370056
:1073240069003700680037006700370066003700df
:1073340065003700640037006300370062003700df
:1073440061003700600037005f0037005e003700df
:107354005d0037005c0037005b0037005a003700df
:1073640059003700580037005700370056003700df
:1073740055003700540037005300370052003700df
:1073840051003700500037004f0037004e003700df
:107394004d0037004c0037004b0037004a003700df
:1073a40049003700480037004700370046003700df
:1073b40045003700440037004300370042003700df
:1073c40041003700400037003f0037003e003700df
:1073d4003d0037003c0037003b0037003a003700df
:1073e4001b003700380037003700370036003700fd
:1073f40035003700340037003300370032003700df
:1074040016003700300037002f0037002e003700f9
:10741400150037002c0037002b0037002a003700f6
:1074240029003700280037001200370026003700f3
:107434001c0037001e0037002300370022003700ed
:10744400210037000e003700130037000f0037000b
:107454000040eb00004f78001b00370010c0b30061
:10746400004f78001800370020c0b300004f7800a8
:107474001500370030c0b300004f78001200370009
:1074840040c0b300004f78000f00370050c0b30075
:10749400004f78000c00370060c0b300004f780044
:1074a4000900370070c0b300004f780006003700b1
:1074b400f0ceb300004f780003003700f0cdb300e6
:1074c400004f7800000000001e407800ea4f500092
:1074d40004003a008040eb0000ccb30047ff0700f3
:1074e400030037001e40780011c0b30043ff0700bb
:1074f4001e0090000000e800100798001e00900095
:10750400104078000004e00076ff3a000080fa00a2
:10751400000006000200fa008040eb0000c4b30043
:1075240036ff07000000eb00000f7800060037006c
:1075340040662b001e0040001040780011c0b300cc
:107544002eff07001e0fe800f00320009e007800c5
:10755400808f5000f6ff34008040eb0000c8b30079
:0c75640026ff07000080fa00000006006f
:020000040000fa
:107570000a080000500000000000000000080000a1
:1075800008000000000000000808000002000000e1
:107590000000000078080000100000000200000059
:1075a000494e460000696e0066004e00414e0000e4
:1075b0006e616e00000000005a0800001e0000000e
:1075c00002000000286e69006c2900002500680098
:1075d000076c09004c836a009074a0007ac0000018
:1075e0008068880000846c008200810088080000a8
:0c75f0000200000000000000000000008d
:020000040000fa
:1075fc00f03fb1000180b10006003500ee03090038
:10760c0000000000403fb1000180b100fbff3d00d5
:10761c001000b000203fb0000200350000800900cf
:08762c00000000000000060050
:020000040000fa
:020000040005f5
:0457f400ffff0000b3
:020000040000fa
:020000040005f5
:0457f800b6230000d4
:020000040000fa
:020000040005f5
:0457fc006f3e0000fc
:00000001FF
